:107000004BC0000064C0000062C0000060C000000F
:107010005EC000005CC000005AC0000058C0000004
:1070200056C0000054C0000052C00000C9C4000097
:107030004EC000004CC000004AC0000048C0000024
:1070400046C0000044C0000042C0000040C0000034
:107050003EC000003CC000003AC0000038C0000044
:1070600036C0000034C0000032C0000030C0000054
:107070002EC000002CC000002AC0000028C0000064
:1070800026C0000024C0000022C0000020C0000074
:107090001EC000001CC0000011241FBECFEFD4E0B2
:1070A000DEBFCDBF11E0A0E0B1E0ECE6FDE702C03D
:1070B00005900D92AC36B107D9F711E0ACE6B1E01E
:1070C00001C01D92AA38B107E1F788D34DC698CF09
:1070D00014BC15BCAA9A589A81E085BF15BE0895C4
:1070E00091E080E80FB6F89480936100909361007E
:1070F0000FBE95BF82E085BF5898509A589A83E298
:1071000084BD8FEF88BD10927F0183E085BD5798C5
:107110005F9A80EE9EE20197F1F70895982F15C0CF
:107120008091F200882371F48091E8008B7F809336
:10713000E80003C08EB3882351F08091E80082FFFD
:10714000F9CF02C08091F1009150992349F7089539
:1071500020917B0130917A018091790190917801A1
:1071600080936D0190936E01C90180936F0190939C
:10717000700108951F93DF93CF9300D000D000D00B
:10718000CDB7DEB7809173018823D9F08091760165
:10719000843049F480917701882339F48091780113
:1071A0008F3F19F40EC0853061F08AE080930001B2
:1071B00083E0809372018091EB0080628093EB000A
:1071C000E3C080917601843009F458C0853030F4F2
:1071D000813059F0833009F0D7C01DC0853009F4E3
:1071E000A0C0863009F0D0C0C3C010917701123022
:1071F00008F0CAC0ADDF112361F480916D01909158
:107200006E0123E0FC0120935700E89507B600FCCF
:10721000FDCF85E008C080917701882311F082308E
:1072200029F496DF89E080930001AEC0813009F037
:10723000ABC020E030E040E050E0F90184918F3FA6
:1072400081F0CA01AA27BB278093710130936E0198
:1072500020936D018AE08093000185E080937201A4
:1072600093C02F5F3F4F4F4F5F4F2030F0E73F07F6
:10727000F0E04F07F0E05F0701F786C080917701EB
:10728000833051F581E080936C0180917C01909175
:107290007D01892B71F080917801813009F074C0F3
:1072A00080917B0190917A01909375018093740194
:1072B0006BC080917801882361F42CE088E190E034
:1072C0000FB6F894A895809360000FBE20936000DD
:1072D0005BC01092010158C0882309F055C080910D
:1072E00078018F3F09F050C0E0E0F0E093E085E0E6
:1072F00090935700E89507B600FCFDCF80935700A8
:10730000E89507B600FCFDCFE058FF4F20E7E030DE
:10731000F20771F781E180935700E89510927301AD
:1073200033C0DE011196E5E0F1E083E001900D92BB
:107330008150E1F7DE011496E2E0F1E083E0019094
:107340000D928150E1F79091780180917701882327
:1073500029F4FE01E90FF11D818107C08130A1F4FC
:10736000FE01BC97E90FF11D808180937E010CC066
:1073700080917701833041F480917801882321F452
:10738000809179018093710126960FB6F894DEBF43
:107390000FBECDBFCF91DF911F9108952F923F92E5
:1073A0004F925F927F928F929F92AF92BF92CF92B5
:1073B000DF92EF92FF920F931F93DF93CF9300D052
:1073C000CDB7DEB7009188011091890110937D013E
:1073D00000937C01809182018F77813209F0EAC1AC
:1073E00080918301833009F4AFC1843030F481305F
:1073F00071F0823009F0DEC112C1853009F4C2C1DA
:10740000853008F4B7C1863009F0D4C1CAC1809173
:10741000E800877F8093E80080916C01882319F051
:10742000A9DE10926C010115110529F42BC08EB351
:10743000882309F4BFC18091E80082FFF8CF8091D2
:10744000F1008093760198012150304030937D0106
:1074500020937C01E7E7F1E00CC08091F10081937B
:107460002150304061E0EC37F60719F43183208376
:1074700008C08091F200882381F730937D0120932A
:107480007C0178DE80910001853009F0C4C08091D4
:107490007C0190917D01892B21F482E08093000191
:1074A000BAC08AE13BDEE0906D01F0906E018E2D56
:1074B0008F7134DE80906F01909070010894811C70
:1074C000911C84010E191F0908948108910880916C
:1074D0007701882309F09AC0C801969587959A8309
:1074E0008983C701A0917101B0E09C01AD0162E008
:1074F000E62EF12C012D112DE20EF31E041F151F97
:1075000059016A0190E077247394B5E0A3E04CC080
:107510008091F200882371F48091E8008B7F809342
:10752000E80004C08EB3882309F444C18091E800C8
:1075300082FFF8CFE981FA813197FA83E98380915C
:10754000F100682F8091F100782FF5010B01709206
:107550005700E89511249F5F903421F029803A80EC
:107560002328A9F4F901B0935700E89507B600FC69
:10757000FDCF29803A80232851F0F701A0935700CE
:10758000E89507B600FCFDCFA801970190E042E026
:10759000242E312C412C512CE20CF31C041D151D02
:1075A000A20CB31CC41CD51C49805A80452809F084
:1075B000AFCF90926E0180926D0181E18093570070
:1075C000E89527C08091F200882371F48091E8004B
:1075D0008B7F8093E80004C08EB3882309F4EAC04F
:1075E0008091E80082FFF8CF6091F10080916D01F9
:1075F00090916E01ABD380916D0190916E010196D7
:1076000090936E0180936D0101501040011511059A
:10761000C9F680E183DD8091E8008B7FBFC0809157
:10762000E800877F8093E80004C08EB3882309F4C4
:10763000C1C08091E80080FFF8CF809100018930BF
:1076400091F08A3069F480917701813049F480911A
:107650006D0190916E018093F1009093F1009BC0B9
:1076600080917E0196C060916F01709170012091B0
:107670006D0130916E016F5F7F4F7B01E21AF30A5B
:107680006150704080917701882389F587011695B4
:107690000795C901A0917101B0E09C01AD011FC027
:1076A0008091F200803271F48091E8008E7F8093A7
:1076B000E80004C08EB3882309F47CC08091E80000
:1076C00080FFF8CFF901859194918093F100909318
:1076D000F100015010402E5F3F4F4F4F5F4F01159B
:1076E0001105F1F670936E0160936D0129C082302F
:1076F00039F523C08091F200803271F48091E80066
:107700008E7F8093E80004C08EB3882309F452C0B2
:107710008091E80080FFF8CF00916D0110916E011B
:10772000C8010CD38093F1000F5F1F4F10936E01BF
:1077300000936D010894E108F108E114F104D1F619
:1077400082E08093000127C08091E800877F8093CA
:10775000E800809172018093F1001092F100109284
:10776000F1001092F100809100018093F1001092DD
:10777000F10011C08091E800877F8093E8001092AB
:10778000720117C08091E800877F8093E8008091A4
:1077900000018093F1008091E8008E7F8093E800E3
:1077A00008C08091E800877F8093E80082E08093A2
:1077B00000018FD00F900F90CF91DF911F910F910B
:1077C000FF90EF90DF90CF90BF90AF909F908F9001
:1077D0007F905F904F903F902F9008951F9384B7B4
:1077E00080938A0184B7877F84BF88E10FB6F894BD
:1077F00080936000109260000FBE72DC4F9B02C04D
:1078000011E027C0CED0789411E019C08ED2AA9B87
:1078100016C0AA9A80917F01882331F088B58F3FE6
:1078200041F410927F0108C088B5882329F4109391
:107830007F0188B58F5F02C088B5815088BD809177
:107840000101882319F780916C018823F9F660D033
:1078500010E03EDC1ABD80918A018BBDE09174017D
:10786000F09175010995FA01923071F0933089F029
:10787000913029F488E091E022E130E015C080E009
:1078800090E020E030E010C08AE191E02BE130E0B0
:107890000BC0882329F485E391E024E030E004C0A4
:1078A00089E391E020E330E091838083C90108956A
:1078B0008091EB0081608093EB001092ED0060936B
:1078C000EC004093ED008091EE00881F8827881F10
:1078D00008958091820188238CF403C08EB388239D
:1078E000B1F08091E80082FFF9CF8091E8008B7FB2
:1078F0008093E80008958EB3882349F08091E800D2
:1079000080FFF9CF8091E8008E7F8093E800089592
:1079100051D053D0E0EEF0E0808181608083E8EDCB
:10792000F0E080818F77808319BCE3E6F0E080810E
:10793000816080831092810108953CD03ED0809177
:10794000D800982F9F779093D80080688093D800B4
:107950008091D8008F7D8093D80084E089BD89B55F
:10796000826089BD09B400FEFDCF1EBA109280016D
:1079700080E060E042E29CDF8091E1008E7F8093B6
:10798000E1008091E20081608093E2008091E2005A
:1079900088608093E2008091E0008E7F8093E00019
:1079A0000895E3E6F0E080818E7F808381E080931C
:1079B0008101C3CF1092E20008951092E100089572
:1079C0001F920F920FB60F9211242F933F934F9354
:1079D0005F936F937F938F939F93AF93BF93EF9337
:1079E000FF938091E10080FF16C08091E20080FF4C
:1079F00012C08091E2008E7F8093E2008091E200CD
:107A000080618093E2008091D80080628093D800EA
:107A100019BC1EBA2DD18091E10084FF2DC0809148
:107A2000E20084FF29C084E089BD89B5826089BDF8
:107A300009B400FEFDCF8091D8008F7D8093D800DF
:107A40008091E1008F7E8093E1008091E2008F7E43
:107A50008093E2008091E20081608093E200809157
:107A60008001882331F48091E30087FD02C081E02A
:107A700001C084E08EBBFCD08091E10083FF21C077
:107A80008091E20083FF1DC08091E100877F809399
:107A9000E10082E08EBB109280018091E1008E7F38
:107AA0008093E1008091E2008E7F8093E2008091DC
:107AB000E20080618093E20080E060E042E2F8DE74
:107AC000D7D0FF91EF91BF91AF919F918F917F910F
:107AD0006F915F914F913F912F910F900FBE0F903B
:107AE0001F9018950F931F93DF93CF9300D0CDB7BE
:107AF000DEB78091F100809382018091F100809344
:107B000083018091F1009091F100E4E8F1E080932D
:107B10008401909385018091F1009091F100809310
:107B2000860193838091F1009091F1008093880108
:107B3000958334DC8091E80083FF85C090918201B9
:107B400080918301863091F1873020F4853009F0EF
:107B50007AC007C0883009F449C0893009F073C081
:107B600057C0992309F06FC0109184011F770FB798
:107B7000F8948091E800877F8093E800AADE8091E6
:107B8000E80080FFFCCF8091E3008078812B809318
:107B9000E3008091E30080688093E300112311F4F7
:107BA00082E001C083E08EBB0FBF4DC09058923081
:107BB00008F049C08091840190918501609186010F
:107BC000AE014F5F5F4F4FDEBC01009709F43BC031
:107BD0008091E800877F8093E80089819A8149D06D
:107BE0008091E8008B7F8093E8002DC0903859F594
:107BF0008091E800877F8093E800809180018093E6
:107C0000F1008091E8008E7F8093E80062DE1BC067
:107C10009923C9F4909184019230A8F48091E800EE
:107C2000877F8093E8009093800153DE80918001EC
:107C3000882331F48091E30087FD02C081E001C018
:107C400084E08EBB15D08091E80083FF0AC080914C
:107C5000EB0080628093EB008091E800877F809347
:107C6000E8000F900F90CF91DF911F910F91089531
:107C700008959C014091880150918901461757074A
:107C800018F4F90190E03CC06115710511F0AB01E9
:107C9000F8CF8091E8008E7F8093E80040E050E0CC
:107CA000F0CF8EB38823E9F18530E9F18091E800C7
:107CB00083FF02C081E008958091E80082FD2BC01F
:107CC0008091E80080FF1CC08091F200282F30E0F6
:107CD00007C081918093F100415050402F5F3F4F8A
:107CE0004115510519F02032310598F390E020320A
:107CF000310509F491E08091E8008E7F8093E800DF
:107D00004115510571F6992361F605C08EB388239C
:107D100041F0853041F08091E80082FFF7CF80E0AC
:107D2000089582E0089583E008958EB3882329F0B2
:107D30008091E80083FF01C0D5CE0895F999FECF68
:107D400092BD81BDF89A992780B50895262FF9999B
:107D5000FECF1FBA92BD81BD20BD0FB6F894FA9A2E
:0C7D6000F99A0FBE01960895F894FFCF29
:107D6C0002011E958A20DCFB12011001000000208C
:107D7C00EB03F02F00000001000109021B000101C0
:107D8C000080320904000000FE01020009210300FA
:107D9C0000000C00010403090430034D0054002DB5
:107DAC0000440042002D00550032002000440046E3
:107DBC00005500200042006F006F0074006C006FD3
:0C7DCC000061006400650072000000000F
:040000030000700089
:00000001FF
